:020000020000FC
:020000000DC031
:020008009EC098
:10001A009AC00FEF07BB0FEF08BB03E301BB0CE06D
:10002A0002BB0FED0DBF02E000BF04E003BF05E213
:10003A0006BF00E00FBD0CE00EBD0DE30BBD08E0EE
:10004A000ABD01E409BF00E205BF00E808B900E003
:10005A0010E02CE330E040E050E060E070E080E047
:10006A0078948895FECF0CE002BB113031F0123043
:10007A0051F0133071F0143099F0032F17D008BBE8
:10008A000DE002BB0895042F11D008BB0EE002BB9D
:10009A000895052F0BD0005808BB0CE102BB089548
:1000AA00062F04D008BB0CE202BB0895003091F081
:1000BA00013091F0023091F0033091F0043091F068
:1000CA00053091F0063091F0073091F0083091F048
:1000DA00093091F000EC089509EF089504EA0895B3
:1000EA0000EB089509E9089502E9089502E80895E0
:1000FA0008EF089500E8089500E9089533953A3025
:10010A0081F430E04395463061F440E053955A302B
:10011A0011F450E06395543021F4623011F450E048
:10012A0060E00895F3DF089533953A3029F430E01A
:10013A004395463009F440E02CE308952A9511F4DA
:10014A00DDDF2CE318958FDF1A9511F414E001D046
:10015A001895803009F08A9500B30C70701751F029
:10016A00803041F402FF03C003FF03C003C0DADF9B
:10017A0001C0DADF702F02FF85E003FF85E00895F2
:00000001FF
